:030000000210FCEF
:03000B000200A54B
:03002B000202AB23
:03005B0002045C40
:030073000204364E
:1000800002030406080C10182030406080040608A3
:100090000C10182030406080A0C00D0D0403060D28
:1000A0000502030202C2AFC0D0C0E020620C20688B
:1000B00002419A306602415AE47385258AC262E59C
:1000C00025F470022121206802210E758B00D0E0FA
:1000D000D0D0D297D295D293D2AF32D297D295D2F6
:1000E000937401D5E0FDE53C1420E21520E10D20DC
:1000F0007D02D294307D02D29602011ED29202017C
:100100001E207D02D296307D02D29402011E758B94
:1001100000D0E0D0D0D297D295D293D2AF32758BA7
:1001200000D0E0D0D0D2AF32419AE525600A207DE0
:1001300002C297307D02C295D293419AE5256002B2
:10014000C293207D02D295307D02D297419AE52557
:10015000600A207D02C295307D02C297207D02D2C6
:1001600097307D02D295419A207D02C296307D0261
:10017000C294207D02C294307D02C2967419D5E0EB
:10018000FDE525600A207D02C297307D02C295D22E
:1001900093419A207D02C296307D02C294C292742D
:1001A00019D5E0FDE525600A207D02C297307D0269
:1001B000C295D293419AC292207D02C296307D02AE
:1001C000C2947419D5E0FDE5256002C293207D023A
:1001D000D295307D02D297419AC292207D02C2947C
:1001E000307D02C2967419D5E0FDE5256002C29308
:1001F000207D02D295307D02D297419A207D02C2A5
:1002000094307D02C296C2927419D5E0FDE5256056
:100210000A207D02C295307D02C297207D02D297CE
:10022000307D02D295419A207D02C294307D02C277
:1002300096207D02C296307D02C2947419D5E0FDED
:10024000E525600A207D02C295307D02C297207D9F
:1002500002D297307D02D295419A30723DE53C2022
:10026000E21A20E129207D02C296307D02C294204C
:100270007D02C294307D02C29602029A20E1E620FD
:100280007D02C296307D02C294C29202029AC2924C
:10029000207D02C294307D02C296E525F4F58A7570
:1002A0008B00D262D0E0D0D0D2AF32C2AFC2AD5359
:1002B000E6EFC0D0C0E0D2D3D2AFC2CEE52960070E
:1002C0002074461529610978007900E580307E01A7
:1002D000F430E50278FF53DACF207E0343DA203092
:1002E0007E0343DA10C2D8C271E580307E01F4305B
:1002F000E50279FFC3E89970CE306103752940208B
:1003000074037529408859D270E52A6004152A6162
:100310001920740543DA01C2D82070026141A8593E
:10032000206102C270207402612A882230690AC3E7
:10033000E522955E4003855E227882B6040385221D
:1003400024C3E52594404002D26420CF0CD0E0D0F5
:10035000D0C2D343E610D2AD32C2CF7802E52960D5
:10036000053074021529C3E55994014005755C00F8
:100370006183755D00756400E55C2401F55C5003E4
:10038000755CFF7982B7020EE547601EC3E52294D3
:100390003240178546227982B7030FE547600BC3C9
:1003A000E52294324004798E8722C3E523952260AA
:1003B000084004152361B90523D8C80564E56470B5
:1003C000021564D565647565017805C3E5649566B5
:1003D0004058C3E5649567500878017565030203CA
:1003E000EDC3E564956850057801756501C3E55F67
:1003F0009524401F7982B70402811FE54770148558
:10040000245FE56404600385666475650175233CBB
:1004100002042AE55F285005755FFF811FF55FE53F
:100420005F047006755DFF7564FFD0E0D0D0C2D365
:1004300043E610D2AD32C0D0C0E0C2AF53917F537B
:10044000E67FC260759100C3E49550F594E4955140
:10045000F595759104D0E0D0D0D2AF32C2AF53E65B
:10046000EFC2ADC0D0C0E0C0F0D2D3D2AFA8FBA9DC
:0E047000FCC2D830710281C353DACF207E0364
:10047E0043DA10307E0343DA20D271E580307E01FC
:10048E00F420E502819A88268927C19A53DACF2073
:10049E007E0343DA20307E0343DA10C2D8C27130B5
:1004AE007402C1867800E580307E01F430E502C129
:1004BE00868859C16D53DACF207E0343DA20307E11
:1004CE000343DA10C271206102A19353DACF207E6A
:1004DE000343DA10307E0343DA20C2D8D271885437
:1004EE008955C3E89552F8E99553F9E4FB7E027AF3
:1004FE0000C3E8948CE994005005755800A183C39D
:10050E00E894C8E994005008E4D2E4FB7A0AA160AA
:10051E00C3E89468E994015008E4D2E3FB7A0FA192
:10052E0060C3E894D0E994025008E4D2E2FB7A1E4C
:10053E00A160C3E894A0E994055008E4D2E1FB7AE7
:10054E003CA160C3E89498E994085008E4D2E0FB1B
:10055E007A787E00C3E89556FCE99557FD30E7089A
:10056E00ECF42401FCEDF4FD755800C3EC9AED9EFD
:10057E00500375580188568957A854A95588528931
:10058E00537802C16DC3E89526F8E99527F9307CBA
:10059E0002C151307B02C151307A02C14A2075022C
:1005AE00A1B6E9FDE8FCA1D5E9C313F9E813F830CB
:1005BE007902C14AE9C313F9E813F8307802C14A47
:1005CE00E9C313FDE813FC206126C3EC941CED94E3
:1005DE00024002A1ECED7018C3EC94C8501205282D
:1005EE00C3E528940A5002C186755900D270C1869F
:1005FE00E528600215287400207F037896E624FA19
:10060E00FEE43400FFC3EC9EFCED9FFD5006780027
:10061E007900C151C3EC94FFED9400400678FF7948
:10062E0000C151EC856FF0A4C5F0A2F733F8790044
:10063E00400302066D78FF790002066DE9C313F9D7
:10064E00E813F8307C0EE9600278FFC3E81338F83F
:10065E00E43400F9C3E894FFE99400400278FF887F
:10066E0059D270206102C186741FF4552F4BF52F9D
:10067E00C274E42B7002D27475294030740375294C
:10068E000A306102C19A20740353DAFE752A2030B3
:10069E007403752A0AD0F0D0E0D0D0C2D3D2AD43C5
:1006AE00E6103279010206CF79030206CF790A02EB
:1006BE0006CF791E0206CF79640206CF79C80206EC
:1006CE00CF7817E4D5E0FDD8FAD9F6227A147B78E4
:1006DE000206F67A107B8C0206F67A0D7BB40206C1
:1006EE00F67A0B7BC80206F6AC257525017902B2A7
:1006FE007DE4C292D5E0FDE5256002C293D5E0FD12
:10070E00D293D5E0FDD292D5E0FDE525600A207D9D
:10071E0002C297307D02C295E570D5E0FD207D02C4
:10072E00D297307D02D2957496D5E0FDD9C1EAF804
:10073E00D5E0FDD8FBDBB1C2928C2522C37C007DB7
:10074E000075F00005F0EA33FAEB33FB50F6EB13CD
:10075E00FBEA13FAC3E9FFE8FEE89AF8E99BF950C1
:10076E0004EFF9EEF8B3EC33FCED33FDD5F0DFED2D
:10077E00F9ECF822E889F08A20D2D4F8A9F07B00AF
:10078E0030F70B7BFFF42401F8E9F43400F9E88527
:10079E0020F0A4ADF0F8E98520F0A4AFF0FEED2E28
:1007AE00F974003FFA7C04C3EA13FAE913F9E8136B
:1007BE00F8DCF48BF030F70AE8F42401F8E9F434AD
:1007CE0000F9E889F0C2D4F8A9F0227882B60403C1
:1007DE0002087BC3E5599419401FE52D5406701984
:1007EE00E547703878057994E7146007780A146045
:1007FE00027812C3E53B984020E547600985615FAA
:10080E007564FF756501852224E4F53EF53FF540DC
:10081E00F541F542F54702087B7547017994E714D7
:10082E007013E523F43333F913F8E9540104F9E8AE
:10083E0054FE02086FE714147014E523F4333333B7
:10084E00F913F8E9540304F9E854FC020877E52398
:10085E00F433333333F913F8E954070404F9E85445
:0E086E00F8C39440F8E99400F9883E893F22CF
:10087C00E547603BC3E53B13F9E53A13F8C3E53EA6
:10088C0098F8E53F99F9500CC3E89480E994FF403F
:10089C00160208B7C3E8947FE9940050030208B726
:1008AC00787F79000208B7788079FF8843894422E1
:1008BC00E5476058E5432540F8E5443541F9854462
:1008CC0020E4300701F43542FA30E709C3EA94F02A
:1008DC0040150208F9C3EA940F50030208F978FF97
:1008EC0079FF7A0F0208F9780079007AF0C3E524D1
:1008FC00955E5006E52460092112E54420E70D21A0
:10090C0012E54430E706884089418A4222E5477067
:10091C000302097D78A1E6FAC3E54333F8E54433D5
:10092C00F9120782E930E70BC3E89480E994FF40A1
:10093C00132154C3E8947FE9940050022154787F2A
:10094C0079002154788079FFE820E715C3E52398D6
:10095C00F84009C3E89401400302097B78010209BD
:10096C007BE8F424012523F8400302097B78FF88F7
:10097C004522E54770030209E078A2E6FAA841A9EE
:10098C0042120782E930E70CC3E89401E994FF4076
:10099C00160209B7C3E894FFE9940050030209B7A3
:1009AC0078FF79000209B7780179FFE920E715C3D0
:1009BC00E54598F84009C3E8940140030209DE7844
:1009CC00000209DEE8F424012545F840030209DEA3
:1009DC0078FF88242278FFC264E52D5406702FD24C
:1009EC0064C3E53B940A4009C3E52594405002C218
:1009FC0064E53B601974FF853BF0848537F0A4F8FF
:100A0C00C5F0600278FFC3E895615002A861886068
:100A1C00227883E6F520120F1D75E8901206B17549
:100A2C00E890E5E820ECFBA8BDA9BE120F9D756B04
:100A3C0055756C00C3740013FD745513FC74552C60
:100A4C00FC74003DFDECFAEDFBC3E89AE99B401405
:100A5C00E56B2455F56BE56C3400F56CEA2CFAEB80
:100A6C003DFB80E5AE6BAF6CC3E56C13F9E56B1326
:100A7C00F8C3E913F9E813F8E56B28F569E56C3967
:100A8C00F56A7A03C3E913F9E813F8DAF7AA201A1E
:100A9C007009756B00756C00020AB71AEA6008EEF3
:100AAC0028FEEF39FFDAF88E6B8F6C2275E89022F6
:100ABC007883E6FFE5E820ECF7A8BDA9BE056DC379
:100ACC00E56D94084052756D00E9FA79A0E7604431
:100ADC00EA7007E56E601B020AF2C3E8956E6010BF
:100AEC00E56E5006600C14020AFE0460F9020AFE60
:100AFC00E56EF56EC3946D401B755EC0C3940440E7
:100B0C0013755E80C39404400B755E40C39404401F
:100B1C0003755E0075BB0822EFC39401601BC3E82C
:100B2C0094FFE994035012C3E8956BE9956C500956
:100B3C00E55E600C155E020B4CE55EF46002055E32
:100B4C00A85EC3E524985002A824C3E8955F400A28
:100B5C00A85FE55FF46003855F5E8825E56DB407EB
:100B6C000375BB1022743279A387F0A4C5F0A2F7E9
:100B7C0033F8C3E8955E4002A85E88228824882555
:100B8C00886122753A00753B7F2275C820A8CCA9D4
:100B9C00CD75C824AA38AB3988388939C3E89AF896
:100BAC00E99BF9AA3AAB3BAC3AAD3B7E047F02C35E
:100BBC00EB940440021E1FC3EB940840021E1FC39B
:100BCC00ED13FDEC13FCDEF7C3EA9CFAEB9DFBEF97
:100BDC006009C3E913F9E813F8DFF7EA28FAEB39EF
:100BEC00FB8A3A8B3B400122753AFF753BFF223062
:100BFC00600261FB854C50854D51D26043E68022EA
:100C0C007892E6FFC3E535948240010FC3E5359435
:100C1C00A040010FC3EF940640027F057E021E30F8
:100C2C0072010EC3E53B940350060E0E3072010E9A
:100C3C00C3E53B940250060E0E3072010EA93BA880
:100C4C003A7A04C3E913F9E813F8DAF7C3E89EF823
:100C5C00E99400F94009C3E89402E994005004783F
:0E0C6C0002E4F9E9FBE8FAC3E913FDE813FC22
:100C7A00884C894DC3EF94036037EF20E00DE82CD0
:100C8A00F8E93DF9ECFAEDFB020CA8E828F8E93995
:100C9A00F9C3E89402F8E99400F97A02E4FBC3EF95
:100CAA009403400D8A4E8B4F884889498C4A8D4B54
:100CBA0022884E894F8A488B498C4A8D4B22306054
:100CCA000281C8D26043E680E52D54066027A83A1F
:100CDA00A93BE53494085006E820E002A94D759135
:100CEA0000C3E498F594E499F595759104D260539C
:100CFA00917F43E68022D265753D00752000020D82
:100D0A0013D265753D00752040E52D54066002C278
:100D1A0065D2AF206005E53D60012278017A02C301
:100D2A00E53B940540027802C3E53B940A40027809
:100D3A0003C3E53B940F40027A03306904781E7AB4
:100D4A0001206007E53D6003D2AF22D2AF0000C2A6
:100D5A00AFC3E53BFB940F40027B0FEB04307301FA
:100D6A002320620123F93069027982E58BC3994015
:100D7A00D0053DEAFBE59B5440B52004DBF7A1AE64
:100D8A00206502A113C265759100AE3AAF3BC3E478
:100D9A009EF594E49FF595759104D26053917F4333
:100DAA00E680A113306502A113D896D2AF2230692A
:100DBA000B0534206016753400020DD620600D2014
:100DCA00650A206B07158115810215B822A84EA95C
:100DDA004F75910053917FC3E498F594E499F59582
:100DEA00759104854850854951D26043E68022783E
:100DFA00003064053065027801E53575F007A4F91D
:100E0A00E5F028F5F0E9A2F013A2F113A2F213F526
:100E1A0035C394785003753578C3E535953640085F
:100E2A00D266D297D295D293306002C132854A50A7
:100E3A00854B51D26043E68022C2AFC296C294C2A9
:100E4A009230720B9001FC7419D5E0FD020E592004
:100E5A007D02D296307D02D294759F13753C0202B0
:100E6A000F98C2AF207D02D295307D02D2973072A0
:100E7A00179001D9C292207D02C294307D02C29697
:100E8A007419D5E0FD020E9590013C306206E52505
:100E9A006002C293207D03759F10307D03759F11F8
:100EAA00753C03020F98C2AFC296C294C2923072C6
:100EBA000B9001B67419D5E0FD020EC6207D02D250
:100ECA0094307D02D296207D03759F11307D037583
:100EDA009F10753C04020F98C2AFD29330721790DC
:100EEA000193207D02C296307D02C294C292741987
:100EFA00D5E0FD020F0390012A30620EE525600A53
:100F0A00207D02C297307D02C295759F13753C05FC
:100F1A00020F98C2AFC296C294C29230720B90016D
:100F2A00687419D5E0FD020F33D292207D03759FB4
:100F3A0010307D03759F11753C06020F98C2AF20D1
:100F4A007D02D297307D02D29530721F90022720FF
:100F5A007D02C296307D02C294207D02C294307D09
:100F6A0002C2967419D5E0FD020F7890014E3062E4
:100F7A000EE525600A207D02C295307D02C29720C7
:100F8A007D03759F11307D03759F10753C01C26604
:100F9A00D2AF22900128D297D295D293C296C29408
:100FAA00C292C2622278807607087607087601081C
:100FBA0076040876FF0876FF08760A08760208762D
:100FCA0001087601788C76010876000876B40876EE
:100FDA00FF0876FF0876FF0876030876FF08760191
:100FEA000876FF0876250876D00876780876C80845
:100FFA0076040876FF08760108760008767A08767D
:10100A000A087601227887E6FFC2727888C27DE6EE
:10101A0030E102D27DC27E7889E630E102D27EC317
:10102A00EF94026008758E01D27302103C758E002F
:10103A00C273227880E6149000809378A1F67881B2
:10104A00E6149000809378A2F6120F9D227886E625
:10105A001490008D9378A3F6120F9D22789FE6F8DC
:0E106A00700108C3E8941140027811E82828AC
:10107800F5662566256628F56725662828F5682219
:10108800789CE67536FF75370CB402067536A07580
:10109800370AB4030675368275370522227896E634
:1010A800FA7897E6FB307F047A007BFFC3EB9AFC63
:1010B800C3948250027C82756F00056FEC856FF0D7
:1010C800A4C3E5F0948040F222D27F11A51206C095
:1010D8007A007B007C101206B6E5592AFA74003BA8
:1010E800FBDCF37C04C3EB13FBEA13FADCF7FEC268
:1010F8007F11A522E5EF20E6037520000520903F2B
:10110800FFE520146006901DFF146000930460033F
:1011180075EF12C2D353D9BF7581C043FF80120641
:10112800B175EF0243B203E5B3240420E702F5B337
:10113800120F9D7580FF75A40075F1B275D4DF7527
:1011480090A975A5FC75F2FE75D50175A60175E225
:1011580041120FAF1215F378988670C2AF1206CA03
:101168001206DA1206C01206E11206C01206E812CA
:1011780006C01217161206CA1206CA1206C5C2AF50
:10118800E4F8F6D8FD78C879C8308507D9FBD8F7D0
:10119800021C00120FAF1215F3110F113D11571158
:1011A80066118811A411A578988670120F9D75880C
:1011B8005075891275C82475910475D84075A82290
:1011C80075B80275E690759B80759D0075D10E7592
:1011D800BC5875BB0875BA1175E8801206B1D2AF54
:1011E800120A1D43DA01C2D8C2711206CA7530014B
:1011F800D2617B037A0CE55870067A0CDB022186F3
:101208001206C02070022186C270E559C3940240BC
:10121800E3E52F541F855B5AF55BB55AD7DAD7C279
:101228006153DACF207E0343DA20307E0343DA109D
:10123800C2D8C271C2757528001206C5307409C3B8
:10124800E528940A4002D2751206B6780230740274
:101258007800C3E5599840F0C2AF1206DA1206DAF0
:101268001206DAD2AF1206CA7546001206B6788C94
:10127800E6C394015003021347E530C394015003B9
:10128800021347207435C3E55994FF5003021347EE
:10129800C2AF1206EFD2AF1206C5C3E5599401508A
:1012A800EFC2AF1206DA1206BB1206DAD2AF120686
:1012B800C5C3E55994FF40E902179B7F05D27F110A
:1012C800A51206C5C2AFC27F11A5AE59C3E5599490
:1012D8007FD2AF40741206B1C2AF1206EFD2AFDFB1
:1012E800DC11D1C3EE94057897F61206CA121635AA
:1012F80012171E7F0AD27F11A51206C5C2AFC27F80
:1013080011A5AE59C3E559947FD2AF50E61206B184
:10131800C2AF1206DA1206BB1206DAD2AFDFD61156
:10132800D1EE24057896F61206CA12163512174D14
:101338001206C511A5C3E55994FF40F402179BC3D3
:10134800E559954640038559461206C578017988BE
:10135800E7B403027805C3E5599840024173C2AF68
:101368001206EF1206EF1206EFD2AF1206CA753058
:1013780000E4F531F5320531E531F470390532789C
:101388009AE67819146012783214600D787D14602A
:101398000878FA146003753200C3E53298401715CF
:1013A800327531B478998670C2AF1206EFD2AF7831
:1013B8009886701206C51206BBE5297005307402BE
:1013C800218678012074027806C3E5599840A7124F
:1013D80006C5E52970022186C2AF120F9DE4F522E9
:1013E800F523F524F525D2AF78858662F53EF53FDD
:1013F800F540F541F542F56DF547F52CF52DF53538
:10140800120B8F756D0875BB101206B1120AB8E57C
:10141800E820ECFBA8BDA9BEE97001F8886E120AA5
:10142800BC756D0875BB107887E6FE7602110F78DB
:1014380087EEF6C2AF755EFF120B7185225E8522BC
:101448005F852260D2AF752201752401752501855B
:101458005D64756501D268D269753400120F1D127A
:0E1468000F47120B8F120B96120C0C02148100
:10147600120F9D110F756D0075BB08120D0B120D25
:10148600B8120DD71207D9120DF9120E43120B9688
:10149600120BFB120C0C120CC8120D00120DB81216
:1014A6000DD712087C1209E1120DF9120E6C120BFF
:1014B60096120BFB120C0C120CC8120D0B120DB867
:1014C600120DD71208BC120DF9120EB0120B96129D
:1014D6000BFB120C0C120CC8120D00120DB8120DDB
:1014E600D7120919120DF9120EE2120B96120BFB06
:1014F600120C0C120CC8120D0B120DB8120DD712CD
:10150600097E120DF9120F1D120B96120BFB120C0F
:101516000C120CC8120D00120AB8120DB8120DD713
:10152600120ABC120DF9120F47120B96120BFB1280
:101536000C0C120CC830692F206B2C85615E8561FE
:101546005F855D6475650179327A0AC3E534994031
:1015560009C269D26A8A3302156DC3E559940140FE
:10156600030214810215B8306A1B206B18E5331488
:101576007004C26A8176F533C3E5599401400302CB
:1015860014810215B8C3E55C9401400985615F8545
:101596005D64756501C3E55C94FA5016307404E524
:1015A60029600FC3E53B78F0306B027860985002F3
:1015B6008181C2AF120F9D7887E6FE7602110F7801
:1015C60087EEF6E4F522F523F524F525F562C268E3
:1015D600D2AF1206B1120F9D307406E529700221B2
:1015E60086788DE6C39401400241506179901A0DC8
:1015F6007820121677E520B4A50CA3121677E520FD
:10160600B45A03021615120FAF121635021634908D
:101616001A0378807B0A121677A308DBF9901A0F53
:10162600788C7B15121677A308DBF9901A2422C250
:10163600AF1216B6121690901A00740D12167CA3ED
:10164600740212167CA3741312167C901A03788007
:101656007B0A12167BA308DBF9901A0F788C7B1590
:1016660012167BA308DBF91216C91216A7901A24C4
:1016760022E493F622E6438F01538FFD75EF027540
:10168600B7A575B7F1F0538FFE22438F02438F0142
:1016960075EF0275B7A575B7F1901A0DF0538FFC6B
:1016A60022901A0D74A5D17C901A0E745AD17C2200
:1016B6007A3079D07820901A40D177E520F709A3BF
:1016C600DAF7227A3079D0901A40E7D17C09A3DA8A
:1016D600F922AB71A872BB01027980BB0202798143
:1016E600BB03027982BB04027994BB05027983BBF2
:1016F60006027986BB07027992BB08027987BB0985
:1017060002799CBB0A027988BB0B027989E8F72229
:101716007C051206CADCFB22C2AF1206DA1206E10B
:101726001206E81206EF1206BB1206DA1206E112DC
:1017360006E81206EF1206BB1206DA1206E11206D8
:10174600E81206EFD2AF22C2AF1206EF1206E81277
:1017560006E11206DA1206BB1206EF1206E81206B8
:10176600E11206DA1206BB1206EF1206E81206E1CD
:101776001206DAD2AF22AE71AF72C2AF1206DA1219
:1017860006DA1206DA1206BBDEF21206EF1206BB04
:10179600DFF8D2AF22F11EF116F1167571017572DE
:1017A60001757300F17C7C05AD591206CAC3ED952F
:1017B6005970F5C3E5599401400AC3E55994FF40B1
:1017C600320217D7D1D8D135F11EC2AF75EF12F15B
:1017D60016DCD50573C3E5739403500280C6F11673
:1017E6000572E5711490009A93F808C3E572985053
:1017F6000280AEF116F1160571C3E571940C500224
:10180600809C120FAF121635C2AF75EF1212171663
:101A00000D021307070104FFFF0A020101A55A0195
:101A100000B4FFFFFF03FF01FF25D078C804FF01DA
:051A200000FF0A01FFB8
:101A4000235475726E696779323541232020202036
:101A500023424C48454C4923463333302320202031
:101A60002020202020202020202020202020202076
:101C0000C2AFC2D353D9BF7581C043B20343FF8073
:101C1000752438752503B1BF75EF0275E24043F1B5
:101C20002053A4DFD285780379E67C1075220075F5
:101C30002300901DCC7B0675249875250130850204
:101C4000813D208508D8FBD9F9DCF781AD308508C6
:101C5000D8FBD9F9DCF781ADB17FE493A3C39A60D7
:101C6000028126DBDDB171600281267B08E493FAF4
:101C7000A3B152DBF87A30B152752200752300B15E
:101C800071EAFCEBFDC3ED94FE400EB1718A278B27
:101C900028ED30E0048A828B83B1717AC270D8C398
:101CA000ED94FE601050CEBD0022EC600675200061
:101CB0000200008100A827A9280809D804D90281B8
:101CC000C9B175EA89AAF281BB0D8199C3ED94036C
:101CD0005049EDA2E092007AC5C3E5829400E58305
:101CE000941C5093200010438F02438F0175B7A5B9
:101CF00075B7F1F030001FA827A9280809438F0104
:101D0000538FFDD804D902A11689AAE275B7A5752B
:101D1000B7F1F0A3A103538FFC81757AC1BD030C09
:101D2000E493A3FAB136DCF8B12E81758177AA224B
:101D3000AB23B152EBFAEA6222752608C3E52313FE
:101D4000F523E52213F52250066323A0632201D573
:101D500026EAB1BFB1BF75260AEAF4200102D28596
:101D6000300102C285B1BFC3134002C201D526EBC8
:101D700022B175EAFB208502A175308502A17A7532
:101D80002608AE24AF25C3EF13FFEE13FEB1C3B197
:101D9000BFC3EA133085024480FA30E703632201AF
:101DA000C3E52313F523E52213F52250066323A090
:101DB000632201D526D9E52265236523F52222AECB
:101DC00024AF250E0FDEFEDFFCD20122424C486517
:0A1DD0006C6934373132F33006013C
:00000001FF
